:1000000036C056C055C054C053C052C051C050C075
:100010004FC04EC04DC04CC04BC04AC049C08BA25F
:10002000B0B9C2FF010A2A4B7A85FF010203050716
:10003000EEF3F400010203050700070503020100C7
:10004000020407EEF3F4F0000204070007040200C4
:1000500001020306EEF3F4F00001020306000603BA
:1000600002010002030507000704EE000700112447
:100070001FBECFE5D2E0DEBFCDBF20E0A0E6B0E0FE
:1000800001C01D92AD37B207E1F7E1E6F0E0128260
:10009000ABE6B0E08EEF15968C9315978DEF179623
:1000A0008C93108688E58187612C712C91D0C9C111
:1000B000A7CF8150E82FF0E0EC5DFF4FE491E9BD60
:1000C000089520ED37E0019720F0F9013197F1F71D
:1000D000FACF089588EE93E0F4CF81EA87B986ECF1
:1000E00086B9369A0895369A3699FECF85B1089525
:1000F000EDE7F0E01082118212820895CF93C72DB0
:1001000081E0870D8F73782E662D90E08CD16FEF94
:100110008C2F90E0CF9187C1FF920F931F93CF93C5
:10012000DF93F82E0AE610E0C6E7D0E081E0F8128F
:1001300005C0F8016081CE0176D104C0CE016BD13B
:10014000F8018083015011092196CF37D10571F74D
:10015000DF91CF911F910F91FF900895CFDF81E044
:10016000DBCF811102C019BC0895A3CF0F931F9359
:10017000CF93C82F8B01CC2359F081E09ADFC801BF
:10018000A0DF19BCC8019DDFC8019BDFC150F3CFC0
:10019000CF911F910F9108951F93CF93DF938FEA13
:1001A00087B986EC86B910E1C0E0D0E085E090E048
:1001B00088DF99DFC80FD11D1150C1F7CE0124E0AF
:1001C000969587952A95E1F7DF91CF911F91089534
:1001D0008FE384BBB89A81E08ABD83BF8AB580680B
:1001E0008ABD97B388B3292F30E0209530952B7FB7
:1001F000282B28BB712C872D90E00DD1682E8F3FC6
:1002000009F006C1872D91E0970D792E803498F37F
:10021000A5DF809169008F5F90E04BE250E088237A
:1002200099F09A012F5F3F4FF9013197E491A92F7F
:10023000B0E0AD58BF4FEC93EE2319F0922F941B12
:10024000F1CF8150A901EBCF9093600090937C0097
:10025000262D253FC0F480917F0030917E008313CE
:10026000D0C040917D008413CCC02F5F622E29172F
:1002700008F0612C4F5F40937D003F5F30937E001C
:100280008F5F80937F003ADFC62DC53F28F4D0E012
:10029000CD58DF4FC881DC2F10E080917D00803188
:1002A00068F118DF25DFC2E6D0E0E12CF12C01E097
:1002B00081E08E0D9FEFE91AF90A98819F3FA1F026
:1002C0006DE570E053DFF701E559FF4F60808881ED
:1002D0008027888343DF6FE070E080E247DF88811A
:1002E000802788833BDFF6DE219687E0E816F1045D
:1002F000F9F6612CC0917300DC2F81C0CE3E69F409
:1003000008E087E0D6DE81E290E0DBDE19BC83E422
:1003100090E0D7DE0150A9F772C0C33F41F487E0F7
:10032000C8DE8AE090E0CDDE88E0C3DE12C0C03FC8
:1003300091F468EC70E083E019DF84EF91E0C1DEB6
:1003400064EF71E083E012DF68EC70E083E00EDFC1
:10035000C1DEC0DE54C0C43F81F4BFDEC4DE982FCE
:1003600080E0E82FF0E0E25EFF4FE491E91710F43F
:100370008F5FF7CF6DE770E0EACFCE3F81F4612C5D
:1003800010926900EBDE6AEF70E081E0EFDE81E061
:1003900080936900E3DE6AEF70E081E0D8CFCD3F63
:1003A00091F4612C8FEF80936A00D8DE81E081DECA
:1003B00091DE90DE87E07DDEEFDE80936A00CEDEA8
:1003C00089DE88DEF9CF8D2FCCDEE6DE20916A0053
:1003D000821738F01F5F193078F0DD2369F0D150B3
:1003E0000AC090E030E022503109821793071CF4D4
:1003F000DC1708F4DF5F10E084EF91E062DE78DE66
:100400004CCF76DE8091630081113DCF612C3BCFD4
:1004100080E082DEFECEE199FECF9FBB8EBBE09AEC
:1004200099278DB30895262FE199FECF1CBA9FBB63
:100430008EBB2DBB0FB6F894E29AE19A0FBE0196DF
:060440000895F894FFCFBF
:00000001FF
